:10000000F30AE700140C87014307100AF20C2700DB
:10001000100AA702F30C87014307100A150C2700EA
:10002000070214092B0000082200C0081F08E0087E
:10003000C1081F081F081F080F080F080F0807082E
:100040000708070803080308030801080108010856
:100050008A082108C20810080808040802080108D4
:10006000E20841088A082208C308110818080C0889
:1000700006080308E30842088A082308C40813088E
:1000800019081C080E080708E40843088A08240811
:10009000C50817081B081D081E080F08E5084408B6
:1000A0008A0825080708130819081C080E084508BF
:1000B0008A08260806080308110818080C084608CC
:1000C0008A082708040802080108100808084708D9
:1000D000040802080108C6081008100810081808CB
:1000E000180818081C081C081C081E081E081E08F2
:1000F0001F081F081F081E081E081E081C081C08D1
:100100001C08180818081808100810081008E60835
:100110008A082808C7080108020804080808100807
:10012000E70848088A082908C808110803080608CB
:100130000C081808E80849088A082A08C908190894
:10014000130807080E081C08E9084A088A082B0843
:10015000CA081D081B0817080F081E08EA084B08E4
:100160008A082C081C081908130807080E084C08F0
:100170008A082D080C0818081108030806084D08FD
:100180008A082E08040808081008010802084E080A
:10019000040808081008CB08010801080108030832
:1001A000030803080708070807080F080F080F08C7
:1001B000E1081F081F081F080F080F080F0807088D
:1001C00007080708030803080308010801080108D5
:1001D000EB08CC08110800080A0800080408000809
:1001E0000A080008EC08690068006100850C02003C
:1001F00066006602080C0600F20C2700100C2E00A8
:100200002D00010C2C0009090B02E00EC00F430762
:10021000030B0B021F0E8C014307030B09090B0292
:10022000E00E4306430B2A00400F4307290B0B0245
:100230001F0E2A00EF021D0B0E0B01090B02700EA0
:10024000200F43071D0B1F0C4B018A0143071D0B99
:100250000E0B0A02E00F4307330B1F0C4B018C01FE
:1002600043070E0B030B0A02800F43073B0B1F0CC7
:100270004B012F000E0B0A02A00F43070E0B1F0CA1
:100280004B012C00030B370C8B06AB058B046B0664
:100290008B056B01E1074A0BFF0C260046040000AA
:1002A00066065A0B4605000066075A0B49065E0BA8
:1002B0004905690B460549044804690B4806690B62
:1002C0004805AC020D0C8C014307030B010C2C00FC
:1002D000030B060400006606750B060500006607A2
:1002E000750B0906790B0905820B0605090408043C
:1002F000820B0806820B0805010C2E00ED03820B11
:10030000FF0C2D00A604000066068E0BA60500005B
:1003100066078E0BA906920BA9059B0BA605A904DF
:10032000A8049B0BA8069B0BA805010C2E00ED0250
:100330009B0B010C2D00660400006606A70B6605EA
:1003400000006606A70B6906AB0B6905AF0B6605D7
:1003500069046804AF0B6806AF0B6805610B86047F
:1003600000006606BB0B860500006607BB0B89060E
:10037000BF0B8905C40B860589048804C40B880655
:10038000C40B88056C00030B260400006606D00B26
:10039000260500006607D00B2906D40B2905D80BCB
:1003A000260529042804D80B2806D80B2805F30AAB
:1003B0000B022600E106DA0BEE024A0B0D022E00BC
:0203C0000E0B22
:0207FE00700C7D
:021FFE00EA0FE8
:00000001FF
